:100000000C9435000C945D000C945D000C945D0024
:100010000C945D000C945D000C945D000C945D00EC
:100020000C945D000C945D000C945D000C945D00DC
:100030000C945D000C945D000C945D000C945D00CC
:100040000C945D000C945D000C94CB050C94FF05A2
:100050000C945D000C945D000C945D000C945D00AC
:100060000C945D000C945D00650711241FBECFEF5A
:10007000D8E0DEBFCDBF11E0A0E0B1E0E2E1F0E109
:1000800002C005900D92AE31B107D9F711E0AEE193
:10009000B1E001C01D92A03DB107E1F710E0CAE652
:1000A000D0E004C02297FE010E940308C836D107A1
:1000B000C9F70E94B2050C9407080C940000DC01FB
:1000C000FC01672F71917723E1F7329704C07C918F
:1000D0006D9370836291AE17BF07C8F30895282F00
:1000E00080931E0188309CF484E290E0909320017C
:1000F00080931F0185E290E0909323018093220179
:1001000083E290E0909325018093240133C08031F5
:10011000C4F487E290E09093200180931F0188E26D
:1001200090E0909323018093220186E290E09093E7
:10013000250180932401332727FD30952850304036
:1001400019C0883104F58AE290E0909320018093F1
:100150001F018BE290E0909323018093220189E2BA
:1001600090E09093250180932401332727FD30955B
:100170002051304081E090E002C0880F991F2A95FD
:10018000E2F780932101E0912201F0912301808127
:1001900090912101892B8083E0911F01F091200132
:1001A00080819095892380830895CF92DF92EF928A
:1001B000FF920F931F93DF93CF9300D000D0CDB762
:1001C000DEB78C0149835A836B837C836E0108946C
:1001D000C11CD11C88E2E82E81E0F82EC701B801CD
:1001E0000E94BF050F5F1F4FC701B801F601418193
:1001F0000E94BF050F5F1F4FC701B801F601428182
:100200000E94BF050F5F1F4FC701B801F601438170
:100210000E94BF050F900F900F900F90CF91DF912C
:100220001F910F91FF90EF90DF90CF900895CF92A4
:10023000DF92EF92FF920F931F93CF93DF936B01A7
:100240007C01EA0100E0C701B6012AE030E040E0AD
:1002500050E00E94DF07162FC701B6012AE030E008
:1002600040E050E00E94DF07C901DA016C017D0126
:10027000FE01E00FF11D105D10830F5FC114D1046A
:10028000E104F10401F7CE01800F911D8C01FC0106
:100290001082CE010E945F00C801DF91CF911F91B3
:1002A0000F91FF90EF90DF90CF900895CF93DF9361
:1002B000DB010D900020E9F71197A61BB70BEC01AD
:1002C000E881F9810280F381E02DAD010995DF918C
:1002D000CF9108952F923F924F925F926F927F92AB
:1002E0008F929F92AF92BF92CF92DF92EF92FF9246
:1002F0000F931F93DF93CF93CDB7DEB7C053D14099
:100300000FB6F894DEBF0FBECDBFF89415BC14BC79
:1003100010928100109280001092B1001092B000F3
:1003200082E08093B10088E291E060E070E00E949A
:10033000B805813481F488E291E061E070E00E94C8
:10034000B805853541F488E291E062E070E00E94F2
:10035000B8058C3459F188E291E060E070E041E446
:100360000E94BF0588E291E061E070E045E50E94EF
:10037000BF0588E291E062E070E04CE40E94BF05B6
:1003800088E291E063E070E042E10E94BF0588E20C
:1003900091E064E070E040E20E94BF0585E090E0FB
:1003A00040E05BE460E070E00E94D50088E291E00C
:1003B00063E070E00E94B8050E946F0088E291E05F
:1003C00064E070E00E94B805883010F488E003C053
:1003D000893808F088E880930B0190E0959587951F
:1003E00080930C018E010F5F1F4F88E291E065E062
:1003F00070E00E94B805898388E291E066E070E0D1
:100400000E94B805D80111968C9388E291E067E0CC
:1004100070E00E94B805F801828388E291E068E00C
:1004200070E00E94B805D80113968C9349815A81D7
:100430006B817C814093070150930801609309010F
:1004400070930A0181EB91E00E943A067894FE01D4
:1004500035968CE291E0DF019C011D9221503040E5
:10046000E1F78FEF8D838E838FE78F83EE2462E039
:10047000C62E5F0158E0652E712C6C0E7D1E40E586
:10048000342E39E0432E512C4C0E5D1E2AE3D22E21
:1004900092E4292E8CE0882E912C8C0E9D1E01C09A
:1004A000EF2C81EB91E00E94C006892B09F446C233
:1004B00081EB91E00E94F10635E03093B100C3BCBE
:1004C00003B401FCFDCF88871092B20004E010E075
:1004D00081EB91E00E94C006892B61F081EB91E0F5
:1004E0000E94F106F501E00FF11F80830F5F1F4F9F
:1004F0001092B2008091B200803D50F3C092B100E2
:100500008885843209F075C189858D3409F071C1FF
:100510008A858C3309F06DC10A0D1B1DD8011C9210
:100520008B85803509F445C0813520F4823409F08B
:10053000D1C007C0823509F468C0873509F0CAC048
:10054000A7C0F40120E030E040E050E01FC0DA0135
:10055000C901880F991FAA1FBB1F13E0220F331F69
:10056000441F551F1A95D1F7280F391F4A1F5B1FCB
:10057000862F992787FD9095C097AA2797FDA0956C
:10058000BA2F280F391F4A1F5B1F319660816623DF
:10059000F1F6283010F488E004C0822F293808F0E2
:1005A00088E880930B0190E09595879580930C01E6
:1005B00091C0F40120E030E040E050E01FC0DA01DB
:1005C000C901880F991FAA1FBB1F03E0220F331F09
:1005D000441F551F0A95D1F7280F391F4A1F5B1F6B
:1005E000862F992787FD9095C097AA2797FDA095FC
:1005F000BA2F280F391F4A1F5B1F3196608166236F
:10060000F1F6822F0E946F0065C0F40120E030E017
:1006100040E050E01FC0DA01C901880F991FAA1FEE
:10062000BB1F73E0220F331F441F551F7A95D1F76C
:10063000280F391F4A1F5B1F862F992787FD90952A
:10064000C097AA2797FDA095BA2F280F391F4A1FD8
:100650005B1F319660816623F1F62093070130938A
:1006600008014093090150930A0120583542404047
:10067000504060F480E895E2A0E0B0E0809307018C
:1006800090930801A0930901B0930A0111E023C0DF
:1006900088E291E063E070E040911E010E94BF0596
:1006A00088E291E064E070E040910B010E94BF0598
:1006B00040910701509108016091090170910A0170
:1006C00085E090E00E94D50081EB91E060E071E070
:1006D0000E94560110E0F301308260911E017727DD
:1006E00067FD7095872F972FA2010E941701FC01CB
:1006F000D0822182329660910B0170E080E090E020
:10070000AF010E941701FC01D08222E521833296BD
:1007100060910701709108018091090190910A018F
:10072000AF010E941701DC01FC01D19211963C92AD
:10073000119739E431838EE4828393E59383D482E5
:1007400016962C921697179660E070E080E090E085
:10075000AD010E941701DC01FC01D19283E41196E6
:100760008C93319668E070E080E090E0AF010E94E9
:100770001701DC01FC01D19284E411968C9331962F
:1007800060E170E080E090E0AF010E941701FC01A1
:10079000D082118281EB91E0B3010E94560181EB7E
:1007A00091E06AE00E942C07112309F47ACE81EBD4
:1007B00091E00E941A07A5E0A093B1001092B20048
:1007C0008091B200803DE0F31092B2008091B200BF
:1007D000803DE0F3C092B1004091070150910801C3
:1007E0006091090170910A0181EB91E00E943A0643
:1007F00058CEE0911F01F09120018081909121015C
:10080000892B8083C3BC03B401FCFDCF30910C0164
:1008100040E050E0F501E40FF51F8081A1E060E0C9
:1008200070E0E82EFF248A2F90E08E219F212091F6
:100830002101E0912201F0912301892BF1F08081C7
:10084000822B80831092B20090910B018091B200B4
:100850008917E0F3E0912201F091230190818091CA
:1008600021018095982390831092B20090910B0102
:100870008091B2008917E0F338C08081822B808399
:100880001092B2008091B2008317E0F3E091220150
:10089000F09123019081809121018095982390838C
:1008A0001092B2008091B2008317E0F3E091220130
:1008B000F0912301808190912101892B80831092F6
:1008C000B2008091B2008317E0F3E0912201F09131
:1008D000230190818091210180959823908310922B
:1008E000B2008091B2008317E0F3AA0F6F5F7F4FD1
:1008F0006830710509F097CF4F5F5F4F4017510780
:100900000CF488CFE0912201F09123018081909135
:100910002101892B80831092B2008091B20083174D
:10092000E0F3E0911F01F09120019081809121017D
:10093000809598239083EE24E394B3CDE091240135
:10094000F0912501F08080912101F822EE2009F03C
:10095000A7CDFF2009F4A4CDC3BC03B401FCFDCF97
:1009600040E0282F332727FD30951092B20005C0B4
:100970008091B2008B3F08F093CD808190E082237C
:100980009323892BA9F71092B20005C08091B20081
:100990008B3F08F085CD808190E082239323892BC3
:1009A000A9F34F5F493009F71092B20005C080915A
:1009B000B2008B3F08F074CD808190E082239323B6
:1009C000892BA9F71092B20005C08091B2008B3F2D
:1009D00008F066CD808190E082239323892BA9F3D0
:1009E0001092B20005C08091B2008B3F08F058CD44
:1009F000808190E082239323892BA9F78091B20014
:100A00008093270190E09C013595279595958795D2
:100A100095958795082F020F00932601A091240138
:100A2000B091250180912101282F332727FD309592
:100A30001092B20005C08091B2008B3F08F030CD1B
:100A40008C9190E082239323892BA9F31092B2001A
:100A500005C08091B2008B3F08F022CD8C9190E0D0
:100A600082239323892BA9F78091B200081700F302
:100A70001092B20005C08091B2008B3F08F010CDFB
:100A80008C9190E082239323892BA9F31092B200DA
:100A900005C08091B2008B3F08F002CD8C9190E0B0
:100AA00082239323892BA9F743E050E010E060E014
:100AB00070E01092B20005C08091B2008B3F08F048
:100AC00049C08C9190E082239323892BA9F3109243
:100AD000B20004C08091B2008B3FE0F58C9190E0B1
:100AE00082239323892BB1F78091B200081710F469
:100AF00081E01BC01092B20004C08091B2008B3F15
:100B000048F58C9190E082239323892BB1F31092C6
:100B1000B20004C08091B2008B3FE0F48C9190E071
:100B200082239323892BB1F780E090E0062E02C048
:100B3000880F991F0A94E2F7182B6F5F7F4F683078
:100B4000710509F0B6CFF501E40FF51F10834F5F73
:100B50005F4FACCF4350504081EB91E0B3010E9416
:100B6000B5079ECC80E00E946A0180E090E0089585
:100B7000F999FECF72BD61BDF89A80B50895F999D3
:100B8000FECF1FBA72BD61BD40BD0FB6F894FA9A90
:100B9000F99A0FBE08951F920F920FB60F9211246B
:100BA0002F933F934F938F939F93EF93FF93409196
:100BB000C6002091690130916A012F5F3F4F2F736A
:100BC000307080916B0190916C012817390759F0B2
:100BD000E0916901F0916A01E75DFE4F4083309337
:100BE0006A0120936901FF91EF919F918F914F913D
:100BF0003F912F910F900FBE0F901F9018951F924D
:100C00000F920FB60F9211242F933F938F939F93C0
:100C1000EF93FF932091AD013091AE018091AF0130
:100C20009091B0012817390731F48091C1008F7D70
:100C30008093C10014C0E091AF01F091B001E3597D
:100C4000FE4F20818091AF019091B00101968F738A
:100C500090709093B0018093AF012093C600FF91F4
:100C6000EF919F918F913F912F910F900FBE0F9019
:100C70001F901895AF92BF92DF92EF92FF920F9361
:100C80001F93CF93DF93EC017A018B01DD24403079
:100C900081EE580780E0680780E0780711F0DD24D6
:100CA000D39491E0A92EB12CEC89FD89DD2069F067
:100CB000C5010E8C02C0880F991F0A94E2F7808349
:100CC00060E079E08DE390E005C0108260E874E8B0
:100CD0008EE190E0A80197010E94DF07215030408B
:100CE00040405040569547953795279580E12030F4
:100CF000380720F0DD2011F0DD24D6CFE889F9890E
:100D00003083EA89FB892083EE89FF89408121E0D5
:100D100030E0C9010A8C02C0880F991F0A94E2F7DB
:100D2000482B4083EE89FF894081C9010B8C02C0AA
:100D3000880F991F0A94E2F7482B4083EE89FF89B8
:100D40004081C9010C8C02C0880F991F0A94E2F7F8
:100D5000482B4083EE89FF8980810D8C02C0220FD1
:100D6000331F0A94E2F7209528232083DF91CF9147
:100D70001F910F91FF90EF90DF90BF90AF9008957B
:100D8000DC011C96ED91FC911D97E05CFF4F2191D9
:100D9000319180819181281B390B2F733070C901EB
:100DA0000895DC011C96ED91FC911D97E05CFF4FCE
:100DB00020813181E054F040DF01AE5BBF4F8D9167
:100DC0009C9111972817390719F42FEF3FEF07C0AF
:100DD0008D919C91E80FF91F8081282F30E0C90187
:100DE0000895DC011C96ED91FC911D97E05CFF4F8E
:100DF00020813181E054F040DF01AE5BBF4F8D9127
:100E00009C9111972817390719F42FEF3FEF10C065
:100E10008D919C911197E80FF91F20818D919C91E4
:100E2000119701968F73907011969C938E9330E07A
:100E3000C9010895FC0186859785DC01A05CBF4F40
:100E4000FC01EE5BFF4F2D913C91119780819181C8
:100E500028173907C1F70895CF93DF93EC01EE858A
:100E6000FF85E05CFF4F20813181E054F0402F5F2F
:100E70003F4F2F733070DF01AE5BBF4F8D919C9160
:100E8000119728173907D1F3E05CFF4F80819181DA
:100E9000E054F040E80FF91F6083EE85FF85E05CC9
:100EA000FF4F31832083EE89FF89208181E090E02C
:100EB0000D8C02C0880F991F0A94E2F7282B20831B
:100EC00081E090E0DF91CF9108951092B4011092EB
:100ED000B30188EE93E0A0E0B0E08093B501909379
:100EE000B601A093B701B093B80181E191E090936E
:100EF000B2018093B10189E291E09093BE018093A9
:100F0000BD018DE691E09093C0018093BF0185EC17
:100F100090E09093C2018093C10184EC90E09093A3
:100F2000C4018093C30180EC90E09093C60180934C
:100F3000C50181EC90E09093C8018093C70186ECD5
:100F400090E09093CA018093C90184E08093CB0123
:100F500083E08093CC0187E08093CD0185E080938E
:100F6000CE0181E08093CF010895CF92DF92EF927E
:100F7000FF920F931F93CF93DF937C016B018A0144
:100F8000C0E0D0E00FC0D6016D916D01D701ED91A9
:100F9000FC910190F081E02DC7010995C80FD91F80
:100FA000015010400115110571F7CE01DF91CF916D
:100FB0001F910F91FF90EF90DF90CF900895A1E2E5
:100FC0001A2EAA1BBB1BFD010DC0AA1FBB1FEE1FC3
:100FD000FF1FA217B307E407F50720F0A21BB30B0E
:100FE000E40BF50B661F771F881F991F1A9469F78A
:100FF00060957095809590959B01AC01BD01CF01E6
:101000000895EE0FFF1F0590F491E02D0994F894D8
:02101000FFCF10
:1010120073617665643A00004B0000201000000006
:0E102200002C07B507C006F106D1061A07001C
:00000001FF
